:100000000C943E050C9485050C948A060C94850589
:100010000C9485050C9485050C9485050C94850538
:100020000C9485050C9485050C948A0D0C94600E37
:100030000C94141D0C9485050C9485050C94850571
:100040000C9485050C9485050C9485050C94850508
:100050000C9485050C94881D0C9485050C948505DD
:100060000C9485050C9485050C9485050C948505E8
:100070000C9485050C9485050C9485050C948505D8
:100080000C9485050C9485050C9485050C948505C8
:100090000C9485050C9485050C9485050C948505B8
:1000A0000C9485050C9485050C948505D10EF30EF2
:1000B000E10FF30EE10F380F5B0FE10FB00FC30F2D
:1000C000DD12DD120C130C136A13A813C215C2152E
:1000D000C113C215C214C2149615C215C215AD15AE
:1000E00032291E1F20212223242526272D2E2A2BAC
:1000F000141A0815171C180C12132F302878041620
:1001000007090A0B0D0E0F33343579311D1B061903
:100110000511103637387D557A2C393A3B3C3D3E37
:100120003F4041424353475F6061565C5D5E5759B3
:100130005A5B62634648324445677B7F6501020330
:100140005250514F68696A6B6C6D6E6F7071725866
:1001500000494C754A4D734B4E767C777E746654DD
:10016000706275663A2066756C6C0A0025303258EC
:1001700020004B6579626F617264207374617274E0
:100180002E0A0055534220636F6E6669677572656B
:10019000642E0A000D0A696E69740A005B445D00F2
:1001A0005B435D002C035800540020006B00650089
:1001B000790062006F00610072006400200063003B
:1001C0006F006E00760065007200740065007200BA
:1001D00000000E0374002E006D002E006B002E0038
:1001E00000000403090409028D00050100A0320982
:1001F0000400000103010100092111010001224056
:10020000000705810308000A090401000103010237
:1002100000092111010001224D0007058203080099
:100220000A09040200010300000009211101000174
:100230002236000705830308000A090403000203AD
:10024000000000092111010001222200070584039A
:100250002000010705040320000109040400010334
:100260000000000921110100012239000705850362
:100270002000011201100100000008EDFE126501CE
:10028000000102000105010906A101050719E02985
:10029000E715002501950875018102050819012956
:1002A00005950575019102950175039101050719E1
:1002B0000029F71500250195F875018102C0063166
:1002C000FF0974A1010975150026FF009520750826
:1002D00081020976150026FF00952075089102C05D
:1002E00005010980A101850216810026B7001A8147
:1002F000002AB700751095018100C0050C0901A105
:10030000018503160100269C021A01002A9C027531
:100310001095018100C005010902A1010901A10098
:1003200005091901290515002501950575018102A9
:100330009501750381010501093009311581257F7A
:1003400095027508810609381581257F9501750884
:100350008106050C0A38021581257F9501750881F3
:1003600006C0C005010906A101050719E029E71526
:100370000025019508750181029501750881010527
:1003800008190129059505750191029501750391DB
:10039000010507190029FF150026FF0095067508BD
:1003A0008100C0636F6E73756D65723A20253034BD
:1003B000580A0073797374656D3A20253034580AF1
:1003C000000A002530325820006B6579626F617237
:1003D000643A20004C45443A20253032580A002522
:1003E0003032583A202530386225730A00722F6364
:1003F0002030313233343536370A0064656C5F6B38
:1004000065795F6269743A2063616E277420646560
:100410006C3A20253032580A006164645F6B65795C
:100420005F6269743A2063616E2774206164643A84
:1004300020253032580A00290A002575002F002592
:1004400075005D280025640020002564002000253B
:10045000640020002564007C0025303258006D6F58
:100460007573656B6579205B62746E7C782079208A
:100470007620685D287265702F61636C293A205B75
:10048000006D6B5F776865656C5F74696D655F743F
:100490006F5F6D6178203D2025640A006D6B5F778A
:1004A0006865656C5F6D61785F7370656564203D3C
:1004B0002025640A006D6B5F74696D655F746F5F02
:1004C0006D6178203D2025640A006D6B5F6D617859
:1004D0005F7370656564203D2025640A006D6B5F65
:1004E000696E74657276616C203D2025640A006D2A
:1004F0006B5F64656C6179203D2025640A006D6B3B
:100500005F776865656C5F74696D655F746F5F6D5B
:100510006178203D2025640A006D6B5F7768656512
:100520006C5F6D61785F7370656564203D20256444
:100530000A006D6B5F74696D655F746F5F6D6178E4
:10054000203D2025640A006D6B5F6D61785F7370DC
:10055000656564203D2025640A006D6B5F696E74DB
:10056000657276616C203D2025640A006D6B5F64C6
:10057000656C6179203D2025640A000A002575001C
:10058000363A20776865656C5F74696D655F746F76
:100590005F6D61783A20000A00257500353A2077B2
:1005A0006865656C5F6D61785F73706565643A203E
:1005B000000A00257500343A2074696D655F746F18
:1005C0005F6D61783A20000A00257500333A206D8E
:1005D00061785F73706565643A20000A00257500D4
:1005E000323A20696E74657276616C286D73293AAF
:1005F00020000A00257500313A2064656C61792875
:100600002A31306D73293A20000A092D2056616C79
:10061000756573202D0A004D3E004D25643E200077
:100620003F007365742064656661756C740A0043ED
:100630003E200077686572652064656C74613A20BD
:10064000637572736F723D25642C20776865656CE5
:100650003D25640A53656520687474703A2F2F65D0
:100660006E2E77696B6970656469612E6F72672F92
:1006700077696B692F4D6F7573655F6B6579730A69
:10068000000A092D204D6F7573656B6579202D0A61
:100690004553432F713A09717569740A313A0964F7
:1006A000656C6179282A31306D73290A323A0969FB
:1006B0006E74657276616C286D73290A333A096D20
:1006C00061785F73706565640A343A0974696D65B1
:1006D0005F746F5F6D61780A353A09776865656C9C
:1006E0005F6D61785F73706565640A363A09776893
:1006F00065656C5F74696D655F746F5F6D61780AC5
:100700000A703A097072696E742076616C7565734F
:100710000A643A097365742064656661756C747364
:100720000A75703A092B310A646F776E3A092D31D8
:100730000A706775703A092B31300A7067646F77F9
:100740006E3A092D31300A0A7370656564203D20C8
:1007500064656C7461202A206D61785F73706565D3
:1007600064202A2028726570656174202F207469C6
:100770006D655F746F5F6D6178290A003F004D3EC3
:100780002000433E20004C25640A000A092D204326
:100790006F6E736F6C65202D0A4553432F713A09B4
:1007A000717569740A6D3A096D6F7573656B65795A
:1007B0000A000A092D204D61676963202D0A643AF9
:1007C0000964656275670A783A096465627567202D
:1007D0006D61747269780A6B3A09646562756720A5
:1007E0006B6579626F6172640A6D3A09646562755E
:1007F00067206D6F7573650A763A0976657273695D
:100800006F6E0A733A097374617475730A633A09F7
:10081000636F6E736F6C65206D6F64650A302D3485
:100820003A096C61796572302D34284631302D4695
:1008300034290A506175733A09626F6F746C6F6185
:100840006465720A6E3A094E4B524F0A003F004EE1
:100850004B524F3A206F66660A004E4B524F3A2079
:100860006F6E0A0074696D65725F72656164333220
:1008700028293A202530346C580A006B6579626F5C
:100880006172645F6E6B726F3A2025580A006B6567
:1008900079626F6172645F69646C653A2025580AF9
:1008A000006B6579626F6172645F70726F746F6301
:1008B0006F6C3A2025580A00686F73745F6B657916
:1008C000626F6172645F6C65647328293A202558F1
:1008D0000A000A092D20537461747573202D0A00D3
:1008E0004743433A20342E392E32204156522D4C64
:1008F0004942433A20312E382E3073766E204156CD
:10090000525F415243483A2061767235310A004FB6
:100910005054494F4E533A204C554641204D4F5567
:1009200053454B45592045585452414B4559204356
:100930004F4E534F4C4520434F4D4D414E44204E5A
:100940004B524F204B45594D41505F5345435449FD
:100950004F4E20343039360A004255494C443A2033
:10096000366465653731652D646972747920283085
:10097000323A33303A3131204170722032352032F0
:10098000303138290A005649443A203078464545E6
:100990004428742E6D2E6B2E29205049443A203065
:1009A0007836353132285854206B6579626F617220
:1009B0006420636F6E7665727465722920564552A5
:1009C0003A203078303030310A00444553433A20E1
:1009D000636F6E76657274205854206B6579626F10
:1009E00061726420746F205553420A000A092D2059
:1009F00056657273696F6E202D0A000A6D6F7573EC
:100A0000653A206F66660A000A6D6F7573653A2055
:100A10006F6E0A000A6B6579626F6172643A206FCB
:100A200066660A000A6B6579626F6172643A206FCC
:100A30006E0A000A6D61747269783A206F66660A00
:100A4000000A6D61747269783A206F6E0A000A6458
:100A5000656275673A206F6E0A000A6465627567A1
:100A60003A206F66660A000A0A626F6F746C6F61E3
:100A70006465722E2E2E2000433E200011241FBEDE
:100A8000CFEFDAE0DEBFCDBF04B603FE27C0809112
:100A9000CF029091D002A091D102B091D2028730C2
:100AA000904BA740B04BD1F41092CF021092D002DD
:100AB0001092D1021092D20214BE84B7877F84BFF5
:100AC0000FB6F894A89580916000886180936000CB
:100AD000109260000FBEE0E0F8EF099511E0A0E091
:100AE000B1E0EAE2FCE402C005900D92A833B10740
:100AF000D9F722E0A8E3B1E001C01D92AF3CB207F4
:100B0000E1F70E94AE0A0C9413260C940000FF93A8
:100B1000EF93E0913801F0913901309709F0099590
:100B2000EF91FF910895FC018591803011F0EFDF86
:100B3000FBCF0895FF27E0E230E247FF0CC041956C
:100B400097FF09C0EDE26095709580959095611DC5
:100B5000711D811D911D27FF02C0219530E350E2D8
:100B6000AA27660F771F881F991FAA1FA41710F0C6
:100B7000A41B63955A95A9F7AA3008F0A95FA05D58
:100B8000AF93F395611571058105910541F7ED323C
:100B900011F4EF93F395F21718F43F93F395FBCF0D
:100BA0008F91B5DFFA95E1F70895E991F991859173
:100BB000803021F0853219F0AADFF9CF089520E0C6
:100BC000E89455915532C1F3503311F4689455911E
:100BD0005A3348F4505390F3220F022E220F220F63
:100BE000200D250FF4CF0EF421958991999153365C
:100BF00019F3533729F1533559F1BC018827992747
:100C0000E8945C3621F48991999168945591543611
:100C100039F446EF7EF077FF0DC08FEF9FEF0AC0EB
:100C200055374AE039F0583540E121F0523642E07C
:100C300009F00895FF93EF937DDFEF91FF91B7CF18
:100C4000FF93EF93FC0181918030B9F360DFFBCF1C
:100C5000FF93EF9368DFF1CFDF93CF93CDB7DEB78C
:100C60002596A3DFCF91DF910895E9E6F0E080813A
:100C700088608083E9982F98279A2FEF89E698E17A
:100C8000215080409040E1F700C00000279858981C
:100C9000509A5998519A2FEF89EF90E02150804057
:100CA0009040E1F700C000005198599A5098589A26
:100CB000E19AE99A08954FB7F89420913E01309156
:100CC0003F0180913C0190913D014FBF28173907AA
:100CD000F9F09FB7F89420913C0130913D0140918B
:100CE0003E0150913F014217530779F0F901EE0F91
:100CF000FF1FE05CFE4F80812F5F3F4F2F71332736
:100D000030933D0120933C0101C080E09FBF0895D6
:100D100080E008951F920F920FB60F9211240BB628
:100D20000F922F933F934F935F936F937F938F9384
:100D30009F93AF93BF93CF93EF93FF9329B121700C
:100D400090913B01992319F0993058F403C0211177
:100D500008C037C080913A01869521118068809340
:100D60003A0181E0890F80933B01983051F5409121
:100D70003A0150E0CFB7F89480913E0190913F0145
:100D80009C012F5F3F4F2F71332760913C01709181
:100D90003D012617370761F0880F991FFC01E05CC1
:100DA000FE4F5183408330933F0120933E0104C0A6
:100DB00080E691E00E949305CFBF10923B01109214
:100DC0003A01FF91EF91CF91BF91AF919F918F9198
:100DD0007F916F915F914F913F912F910F900BBE3B
:100DE0000F900FBE0F901F9018958D3409F456C0C8
:100DF00000F5883309F462C068F48D3109F45CC0F1
:100E000018F48C31A9F108958533A1F1873309F4E1
:100E100057C008958834E1F130F4863439F18734CD
:100E200009F442C00895893409F442C08B3491F129
:100E300008958B3509F168F48135E1F128F48F3498
:100E4000A9F1803549F10895823551F1833551F189
:100E500008958E35B9F028F48C3581F08D3581F008
:100E600008958F3589F0833689F0089585E50895D2
:100E70008FE608958FE708958AE508958BE5089534
:100E80008CE508958DE508958EE508958FE5089524
:100E900080E6089581E6089582E6089583E6089540
:100EA00081E7089582E7089584E7089585E7089526
:100EB00087E7089588E708958AE708958CE70895FD
:100EC00084E50895CF93DF93D82FD770C82FC695A8
:100ED000C695C6956D2F8C2F0E94661181110DC08D
:100EE000EC2FF0E0EF57FE4F81E090E001C0880F5B
:100EF000DA95EAF79081892B8083DF91CF9108956D
:100F0000CF93DF93D82FD770C82FC695C695C695B7
:100F10006D2F8C2F0E946611882371F0EC2FF0E06A
:100F2000EF57FE4F81E090E001C0880FDA95EAF7B5
:100F30008095908189238083DF91CF91089580915E
:100F4000B10281608093B1020E943506E1E8F1E0D0
:100F500080E18E0F11928E13FDCF0895CF93DF9312
:100F60001F92CDB7DEB70E945B06882309F45CC0F0
:100F70001F928F932CE631E03F932F9389830E9439
:100F80002C060F900F900F900F9090918001898107
:100F9000923081F128F4992341F09130A1F040C0C2
:100FA000933091F19430B1F13BC0803E21F0813E0D
:100FB00031F482E026C081E08093800136C087FF53
:100FC00026C08F772AC0863359F118F48A3229F463
:100FD00027C08A3A29F1863B19F187FD05C00E9496
:100FE000F5060E9462071CC08F770E94F5060E94DA
:100FF000800716C08D3121F08D3991F484E001C055
:1010000083E0809380010EC0853451F485E50E9411
:10101000620708C0853421F485E50E94800702C07C
:101020001092800181E001C080E00F90DF91CF91AC
:101030000895E82FF0E0EF57FE4F80810895E1E832
:10104000F1E080E18E0F11928E13FDCF0895089587
:101050008091B50108959FB7F894109294019FBFB5
:101060009091C602943009F057C09091E9009F70AA
:101070003091EC00232F217030FD20E8922B24E0EA
:101080002093E9002091EB0020FF43C02091EE0067
:1010900027FF3FC020919101222321F02091E800F9
:1010A00025FF37C01092910126E03091E80035FD10
:1010B00015C03091C602343061F53091EB0035FD3A
:1010C00028C0215021F481E08093910122C0EFE9F2
:1010D000FFE03197F1F700C00000E7CF8093F10007
:1010E0008091E80085FD0AC08091E80080FFFCCF78
:1010F0008091E8008E778093E80006C08FB7F8945F
:1011000021E0209394018FBF9F709093E90080E0CD
:1011100008959F709093E9008FEF0895CF93DF9328
:1011200000D01F92CDB7DEB79C018091C6028430FB
:1011300019F593E099833B832A839093E9008FEF1D
:101140009091E800815095FD06C095ED9A95F1F7D4
:1011500000008111F5CF8091E80085FF0DC040E0CF
:1011600050E063E070E0CE0101960E947B0B80911D
:10117000E8008E778093E8000F900F900F90DF913A
:10118000CF910895CF93DF9300D01F92CDB7DEB7F4
:101190002091C602243021F522E029839B838A8393
:1011A00083E08093E9008FEF9091E800815095FDF6
:1011B00006C095ED9A95F1F700008111F5CF809169
:1011C000E80085FF0DC040E050E063E070E0CE0134
:1011D00001960E947B0B8091E8008E778093E80057
:1011E0000F900F900F90DF91CF9108952091C6023C
:1011F0002430F1F422E02093E9002FEF3091E80051
:10120000215035FD06C035ED3A95F1F7000021116A
:10121000F5CF2091E80025FF0BC040E050E065E0ED
:1012200070E00E947B0B8091E8008E778093E8004D
:101230000895CF93DF932091C602243009F048C06F
:10124000EC0180910A018823E1F080910B01882351
:10125000C1F085E08093E9008FEF9091E800815024
:1012600095FD06C09AE29A95F1F700C08111F5CF7D
:101270008091E80085FF2CC040E050E060E270E023
:1012800017C081E08093E9008FEF9091E8008150D2
:1012900095FD06C095ED9A95F1F700008111F5CF07
:1012A0008091E80085FF14C040E050E068E070E005
:1012B000CE010E947B0B8091E8008E778093E8003E
:1012C00080E2FE01A5E9B1E001900D928A95E1F777
:1012D000DF91CF91089580EA91E00E94930580917B
:1012E000C502811109C00E940C0D0E946E0D8091F3
:1012F000E20084608093E20008958CE991E00E940E
:1013000093051092C50208950895209192012F5FD0
:10131000822F62E30E94D925992319F0209392012C
:1013200008951092920180919401882371F1809127
:10133000C602843041F58091E9008F702091EC0065
:10134000922F917020FD90E8892B94E09093E90012
:101350009091EB0090FF14C09091EE0097FF10C0A9
:101360009091E80095FF03C01092F100F9CF9091A1
:10137000E80090FF05C09091E8009E779093E80008
:101380008F708093E90010929401089542E061EC1F
:1013900081E00E94860C42E061EC82E00E94860CB3
:1013A00042E061EC83E00E94860C42E261EC84E062
:1013B0000E94860C42E261EC85E00C94860C8091E0
:1013C000C802833009F455C030F4813071F08230A6
:1013D00009F48EC008958A3009F47AC08B3009F47C
:1013E00060C0893009F09CC020C08091C702813A5A
:1013F00009F096C08091E800877F8093E800809193
:10140000CB029091CC02892B21F460E285E991E036
:1014100003C060E080E090E070E00E94C60B809125
:10142000E8008B778093E80008958091C7028132AD
:1014300009F076C08091CB029091CC02009719F010
:10144000049709F06DC08091E800877F8093E800E1
:101450008091E80082FD05C08091C6028111F8CF1D
:101460005FC08091F1008093B5018091E8008B7797
:1014700053C08091C702813A09F052C08091CB02DB
:101480009091CC02892B09F04BC08091E800877FB6
:101490008093E8008091E80080FFFCCF80910A01F2
:1014A00036C08091C7028132D9F58091CB029091EC
:1014B000CC02892BA9F58091E800877F8093E80012
:1014C0000E94BB0C8091C90280930A010C94E41520
:1014D0008091C702813221F58091E800877F809357
:1014E000E8000E94BB0C8091CA028093B601089567
:1014F0008091C702813AA1F48091E800877F8093B0
:10150000E8008091E80080FFFCCF8091B6018093D5
:10151000F1008091E8008E778093E8000C94BB0C7A
:101520000895089508958091B501809393011092D4
:10153000B50180E00E9427080E941F080C94E41562
:101540000C94930A0E94D31C8091C402882329F032
:101550000E94FC1C81110C94650B089584B7877F51
:1015600084BF0FB6F894A89580916000886180933D
:101570006000109260000FBE90E080E80FB6F89413
:1015800080936100909361000FBE8BE298E00E940F
:10159000A41C84E991E00E9493050E94910A0E9494
:1015A000BA100E940C0D0E946E0D8091E2008460C2
:1015B0008093E20078948091C6028430E1F781ED57
:1015C00097E0019739F0EFE9FFE03197F1F700C0BC
:1015D0000000F7CF83E891E00E9493050E94BC10C1
:1015E00080E091E00E94F90F82E791E00E9493056C
:1015F0000E94920A8091C602853019F40E94A20AC4
:10160000F9CF0E94C010F6CF0E94101D8091930167
:101610008093B50108950C94040B292F33272330B0
:101620003105C9F064F42130310581F022303105F3
:1016300009F043C08DE890E026EE31E042C021324F
:101640003105F1F02232310541F137C082E190E0FD
:1016500023E732E036C099278130910541F082308E
:10166000910541F0892B49F5E2EEF1E005C0E2ED8C
:10167000F1E002C0E4EAF1E0849190E09F0121C032
:101680006530D8F4E62FF0E0EE0FFF1FED5DFE4F62
:101690002081318189E090E014C0653070F470E001
:1016A000FB01EE0FFF1FE75EFE4F20813181FB0142
:1016B000EC5EFE4F808190E004C080E090E020E08E
:1016C00030E0FA0131832083089584E189BD86E109
:1016D00089BD09B400FEFDCF8091D8008F7D809335
:1016E000D8008091E00082608093E0008091E0006B
:1016F00081FDFCCF0895CF92DF92EF92FF920F937E
:101700001F93CF93DF93EC018B016A010E94DA0CE7
:10171000811133C0C114D10439F0F6018081918167
:10172000081B190BC80FD91FE12CF12C011511054D
:1017300019F18091E80085FD16C08091E8008E7750
:101740008093E800C114D10449F0F60180819181B1
:10175000E80EF91EF182E08285E00FC00E94DA0CEB
:10176000882321F30AC089918093F1000150110967
:10177000FFEFEF1AFF0ADACF80E0DF91CF911F91E0
:101780000F91FF90EF90DF90CF9008952091CD02C0
:101790003091CE022617370748F06115710539F4EC
:1017A0002091E8002E772093E80001C0B90140E0C5
:1017B0006115710599F12091C602222309F441C0F7
:1017C000253009F440C02091E80023FD3EC020915F
:1017D000E80022FD30C02091E80020FFE9CF2091F1
:1017E000F2003091F300FC01CF016115710559F051
:1017F0002830310540F481918093F10061507109E6
:101800002F5F3F4FF1CF41E02830310509F040E034
:101810002091E8002E772093E800CACF4111CBCF6A
:101820000AC08091C602882361F0853061F0809102
:10183000E80083FD0AC08091E80082FFF2CF80E0DB
:10184000089582E0089583E0089581E0089520914D
:10185000CD023091CE022617370748F06115710589
:1018600039F42091E8002E772093E80001C0B901F7
:10187000FC0120E06115710581F18091C602882389
:1018800009F43EC0853009F43DC08091E80083FD35
:101890003BC08091E80082FD2DC08091E80080FF70
:1018A000E9CF8091F2009091F3006115710559F034
:1018B0008830910540F424912093F10031966150D5
:1018C00071090196F2CF21E0089709F020E080919C
:1018D000E8008E778093E800CDCF2111CECF0AC0EB
:1018E0008091C602882361F0853061F08091E80024
:1018F00083FD0AC08091E80082FFF2CF80E0089566
:1019000082E0089583E0089581E00895982F97304C
:1019100058F59093E900981739F07091EC002091F8
:10192000ED005091F00003C0242F762F50E021FFEE
:1019300019C03091EB003E7F3093EB003091ED0009
:101940003D7F3093ED003091EB0031603093EB0040
:101950007093EC002093ED005093F0002091EE0086
:1019600027FF07C09F5FD3CF8F708093E90081E08E
:10197000089580E008958091C70287FF11C080918B
:10198000E80082FD05C08091C6028111F8CF11C028
:101990008091E8008B770BC08091C602882349F0C4
:1019A0008091E80080FFF8CF8091E8008E778093E7
:1019B000E80008952091E4003091E50095E640911B
:1019C000EC00842F817040FF22C08091E80080FDF0
:1019D0001CC08091C602882391F0853091F08091DF
:1019E000EB0085FD10C04091E4005091E5004217E6
:1019F000530729F39A01915011F784E0089582E08A
:101A0000089583E0089581E0089580E0089540916D
:101A1000E80042FFDECF08950E947D0D0E94850DF3
:101A2000E0EEF0E0808181608083E8EDF0E080818D
:101A30008F77808319BCA7EDB0E08C918E7F8C935B
:101A400080818F7E80831092C50208950F931F932B
:101A5000CF93DF930E947D0D0E94850DC8EDD0E0ED
:101A600088818F77888388818068888388818F7D4B
:101A70008883E7EDF0E080818068808319BC109254
:101A8000C6021092C2021092C4021092C30200EE6B
:101A900010E0F80180818B7F80838881816088835A
:101AA00042E060E080E00E94860CE1EEF0E08081A0
:101AB0008E7F8083E2EEF0E0808181608083808190
:101AC00088608083F80180818E7F80838881806137
:101AD0008883DF91CF911F910F910895E8EDF0E099
:101AE00080818F7E8083E7EDF0E08081816080835C
:101AF00081E08093C5020C94260DE8EDF0E0808132
:101B00008C7F80831092E20008951092DA00109288
:101B1000E10008951F920F920FB60F9211240BB699
:101B20000F922F933F934F935F936F937F938F9376
:101B30009F93AF93BF93EF93FF938091E10082FF58
:101B40000BC08091E20082FF07C08091E1008B7F93
:101B50008093E1000E9485098091DA0080FF1FC018
:101B60008091D80080FF1BC08091DA008E7F809327
:101B7000DA008091D90080FF0DC084E189BD86E143
:101B800089BD09B400FEFDCF81E08093C6020E94AA
:101B90006B0905C019BC1092C6020E947D09809194
:101BA000E10080FF19C08091E20080FF15C08091A4
:101BB000E2008E7F8093E2008091E200806180935A
:101BC000E2008091D80080628093D80019BC85E043
:101BD0008093C6020E94A00A8091E10084FF30C079
:101BE0008091E20084FF2CC084E189BD86E189BD3B
:101BF00009B400FEFDCF8091D8008F7D8093D8007E
:101C00008091E1008F7E8093E1008091E2008F7EE1
:101C10008093E2008091E20081608093E2008091F5
:101C2000C202882311F084E007C08091E30087FDA1
:101C300002C081E001C083E08093C6020E940B0BCA
:101C40008091E10083FF29C08091E20083FF25C0DD
:101C50008091E100877F8093E10082E08093C6025B
:101C60001092C2028091E1008E7F8093E10080910A
:101C7000E2008E7F8093E2008091E2008061809399
:101C8000E20042E060E080E00E94860C8091F0007B
:101C900088608093F0000E948409FF91EF91BF91CA
:101CA000AF919F918F917F916F915F914F913F91F4
:101CB0002F910F900BBE0F900FBE0F901F90189595
:101CC0001F920F920FB60F9211240BB60F922F9303
:101CD0003F934F935F936F937F938F939F93AF93B4
:101CE000BF93CF93DF93EF93FF93C091E900CF7041
:101CF0008091EC00D82FD17080FDD0E81092E900DF
:101D00008091F000877F8093F00078940E94A80E65
:101D10001092E9008091F00088608093F000CD2B54
:101D2000CF70C093E900FF91EF91DF91CF91BF9108
:101D3000AF919F918F917F916F915F914F913F9163
:101D40002F910F900BBE0F900FBE0F901F90189504
:101D50001F93CF93DF93CDB7DEB7AA970FB6F89452
:101D6000DEBF0FBECDBFE7ECF2E088E08E0F9091B2
:101D7000F10091938E13FBCF0E94DF098091E80060
:101D800083FF1FC18091C7029091C802492F50E084
:101D90004A30510508F015C1FA01EA5AFF4F0C9478
:101DA000F925803881F0823809F00BC18091CB028F
:101DB0008F708093E9008091EB0085FB882780F984
:101DC0001092E90006C08091C3029091C402911163
:101DD00082609091E800977F9093E8008093F100F3
:101DE0001092F100C8C0282F2D7F09F0EAC0882387
:101DF00019F0823061F0E5C08091C902813009F0AC
:101E0000E0C0933009F080E08093C4022BC0809141
:101E1000C902811127C08091CB028F7009F4D1C013
:101E20008093E9002091EB0020FF1CC0933021F447
:101E30008091EB00806214C09091EB0090619093D0
:101E4000EB0021E030E0A90102C0440F551F8A9544
:101E5000E2F74093EA001092EA008091EB0088607C
:101E60008093EB001092E9008091E800877F86C0A4
:101E70008111A7C01091C9021F778091E30080787B
:101E8000812B8093E3008091E800877F8093E800B6
:101E90000E94BB0C8091E80080FFFCCF8091E300A2
:101EA00080688093E300111102C082E001C083E0EA
:101EB0008093C60286C08058823008F082C080912C
:101EC000C9029091CA028C3D53E0950779F583E0F1
:101ED0008A838AE289834FB7F894DE01139620E063
:101EE0003EE051E2E32FF0E050935700E49120FFF1
:101EF00003C0E295EF703F5FEF708E2F90E0EA3005
:101F000010F0C79601C0C0968D939D932F5F24312A
:101F100049F74FBF8091E800877F8093E8006AE22D
:101F200070E0CE0101960E94C60B14C0AE014F5F57
:101F30005F4F6091CB020E940D0BBC01892B09F40D
:101F400040C09091E800977F9093E80089819A8142
:101F50000E94270C8091E8008B778093E80031C0C5
:101F6000803879F58091E800877F8093E800809140
:101F7000C2028093F1008091E8008E778093E800A0
:101F80000E94BB0C1EC081111CC09091C9029230EE
:101F9000C0F48091E800877F8093E8009093C202AC
:101FA0000E94BB0C8091C202811106C08091E300A7
:101FB00087FD02C081E001C084E08093C6020E94D8
:101FC000C6098091E80083FF0AC08091E800877FFE
:101FD0008093E8008091EB0080628093EB00AA96EA
:101FE0000FB6F894DEBF0FBECDBFDF91CF911F912A
:101FF00008959093BC018093BB010895E091BB01CB
:10200000F091BC01309721F00190F081E02D09940E
:1020100080E00895EF92FF920F931F93CF93DF9389
:10202000E091BB01F091BC013097B1F18C010280CD
:10203000F381E02D09958091B10282FF2DC080FFD0
:1020400004C089EC93E00E949305E80110E283EC60
:10205000E82E83E0F82E8091B10280FF0BC08881CA
:102060001F928F93FF92EF920E942C060F900F9079
:102070000F900F90115021961111EDCF8091B10268
:1020800080FF0AC081EC93E0DF91CF911F910F9107
:10209000FF90EF900C949305DF91CF911F910F91DA
:1020A000FF90EF900895E091BB01F091BC01309753
:1020B00021F00480F581E02D09940895CF93DF93FA
:1020C000EC018091B9019091BA01C817D90709F1C3
:1020D000D093BA01C093B901E091BB01F091BC016A
:1020E0003097B9F00680F781E02DCE0109958091F7
:1020F000B10282FF0EC080FF0CC0DF93CF9383EB51
:1021000093E09F938F930E942C060F900F900F9057
:102110000F90DF91CF910895CF93DF93EC018091E1
:10212000B7019091B801C817D90709F1D093B80148
:10213000C093B701E091BB01F091BC013097B9F0B9
:102140000084F185E02DCE0109958091B10282FFD6
:102150000EC080FF0CC0DF93CF9383EA93E09F9380
:102160008F930E942C060F900F900F900F90DF918D
:10217000CF9108950C9465110E943D1D0C949F070A
:10218000BF92CF92DF92EF92FF920F931F93CF9364
:10219000DF9300D000D01F92CDB7DEB70E94AE070C
:1021A0000EEB11E0F12C8F2D0E941908B82EF801CA
:1021B000C080C82639F4F3940F5F1F4FF0E1FF127F
:1021C000F2CF30C08091B10281FD0E948111D12CEB
:1021D000EE24E3948E2D8C21F9F0D982FA8281E0ED
:1021E0009E2D9B2109F480E08B830E94461D816017
:1021F000782F9D838C8349815A816B818D810E94C8
:10220000B71149815A816B817C818D810E94C01CEC
:10221000F80190819E259083D394EE0CF8E0DF12B4
:10222000D9CFC9CF8FEF89838A831B820E94461D35
:102230008160782F9D838C8349815A816B818D8148
:102240000E94B7110E94BF1C0E9407201091BD017F
:102250000E94FE0F181741F10E94FE0F8093BD01EE
:102260009091B10292FF0EC090FF0CC01F928F930D
:1022700084ED93E09F938F930E942C060F900F9014
:102280000F900F908091BD010F900F900F900F90C5
:102290000F90DF91CF911F910F91FF90EF90DF9002
:1022A000CF90BF900C94D11C0F900F900F900F9077
:1022B0000F90DF91CF911F910F91FF90EF90DF90E2
:1022C000CF90BF9008950C9427080895CF93DF9383
:1022D0001F92CDB7DEB769830E94190890E021E014
:1022E00030E0698102C0220F331F6A95E2F728238C
:1022F000392381E0232B09F480E00F90DF91CF9107
:102300000895EF92FF920F931F93CF93DF938DEE7B
:1023100093E00E949305C0E0D0E08DE2E82E81E0DA
:10232000F82E0FED13E08C2F0E9419080E94A91CB3
:10233000FF92EF921F928F93DF93CF931F930F9390
:102340000E942C0621968DB79EB708960FB6F8947A
:102350009EBF0FBE8DBFC031D10529F7DF91CF9150
:102360001F910F91FF90EF90089508950895CF93D6
:10237000DF93CDB7DEB72B970FB6F894DEBF0FBE55
:10238000CDBF942F4F83252F588769877A878B87F6
:102390004A855B85452B21F02F3F09F59F3FF9F4D6
:1023A000DE01119686E0FD0111928A95E9F785E03C
:1023B000FE01379601900D928A95E1F749815A8185
:1023C0006B817C818D819E810E94C1182B960FB6F6
:1023D000F894DEBF0FBECDBFDF91CF9108954F813E
:1023E000588569857A858B850E94C01CD9CFCF938B
:1023F000882309F465C0C82F8CEF8C0F813A20F038
:1024000080E58C0F8E3248F48C2F0E94512381116D
:1024100057C08C2F0E94991B0CC080E28C0F883013
:1024200058F4C77081E001C0880FCA95EAF70E948E
:10243000441CCF910C947E1C8BE58C0F833078F478
:10244000C53A29F0C63A31F083E890E005C081E84A
:1024500090E002C082E890E0CF910C945E1088E595
:102460008C0F853168F5C83A89F0C93A91F0CA3ABB
:1024700099F0CB3AA1F0CC3AA9F0CD3AB1F0CE3AEE
:10248000B9F0CF3AC1F080E090E017C082EE90E062
:1024900014C089EE90E011C08AEE90E00EC085EB8A
:1024A00090E00BC086EB90E008C083EB90E005C0A5
:1024B00084EB90E002C087EB90E0CF910C948C10FD
:1024C000CF910895882349F19CEF980F913A20F01D
:1024D00090E5980F9E3218F40E94EC1B0DC090E21C
:1024E000980F983058F4877091E001C0990F8A9541
:1024F000EAF7892F0E944A1C0C947E1C9BE5980FDA
:10250000933020F480E090E00C945E10885A85317E
:1025100020F480E090E00C948C100895882321F042
:102520000E94441C0C947E1C0895882321F00E9474
:102530004A1C0C947E1C0895BF92CF92DF92EF92BA
:10254000FF920F931F93CF93DF9300D000D000D062
:10255000CDB7DEB725E0FC01DE01119601900D92AA
:102560002A95E1F7FC0140815181028163817481E8
:10257000258122952F706115710509F403C35F3F12
:1025800019F44F3F09F4FEC26C01862F7D836C83E2
:10259000602F782F8D812E830E941D1B182FB92E3E
:1025A0000E941C1B0E940C1AEB2DE295EF70F0E0CC
:1025B000E05AFF4F2E810C94F9258B2D807F9B2DA7
:1025C0009F70F92E882319F0F29490EFF9220023DE
:1025D00049F0FF2009F483C28F2D0E94571C0E94EE
:1025E0007E1C7DC2812F0E946212FF2009F4CAC2A4
:1025F0008F2D0E945D1C26960FB6F894DEBF0FBE8D
:10260000CDBFDF91CF911F910F91FF90EF90DF90A1
:10261000CF90BF900C947E1C8B2D807F9B2D9F7044
:10262000F92E803219F0F29480EFF822112319F07C
:10263000113009F12AC00023B1F08F2D222351F16E
:10264000213041F526960FB6F894DEBF0FBECDBF00
:10265000DF91CF911F910F91FF90EF90DF90CF907E
:10266000BF900C94671C222319F0213009F48AC210
:102670000E946A1C2DC00023F1F0263008F082C2AF
:102680000E94411C8F2129F023C00023F9F0211161
:1026900016C08F2D26960FB6F894DEBF0FBECDBFA5
:1026A000DF91CF911F910F91FF90EF90DF90CF902E
:1026B000BF900C948E12253008F064C209C0F60158
:1026C000858180FF0CC28F708583E3CF21111CC2EE
:1026D0008F2D83C12B2D26952695237030E0211553
:1026E000310521F021303105D1F04CC2002321F019
:1026F000812F9B2D937002C080E090E026960FB64C
:10270000F894DEBF0FBECDBFDF91CF911F910F9127
:10271000FF90EF90DF90CF90BF900C945E1000235D
:1027200021F0812F9B2D937002C080E090E02696CF
:102730000FB6F894DEBF0FBECDBFDF91CF911F91D2
:102740000F91FF90EF90DF90CF90BF900C948C1082
:10275000812F002319F00E948D1E02C00E94F51ED9
:1027600026960FB6F894DEBF0FBECDBFDF91CF9196
:102770001F910F91FF90EF90DF90CF90BF900C943E
:102780007A1F8B2D837009F07BC00111FBC1812F53
:10279000829586958770880F880F912F9F70C92E1C
:1027A000D12CE12CF12C082E04C0CC0CDD1CEE1C2D
:1027B000FF1C0A94D2F714FF12C04FE050E060E013
:1027C00070E004C0440F551F661F771F8A95D2F72B
:1027D000CB01BA01609570958095909503C060E03B
:1027E00070E0CB012B2D269526952370422F50E0CB
:1027F00042305105D9F04330510569F16C297D29EA
:102800008E299F294130510551F126960FB6F89433
:10281000DEBF0FBECDBFDF91CF911F910F91FF9013
:10282000EF90DF90CF90BF900C94311A6C297D29E6
:102830008E299F2926960FB6F894DEBF0FBECDBF16
:10284000DF91CF911F910F91FF90EF90DF90CF908C
:10285000BF900C944B1A0E94311AC701B6012696FC
:102860000FB6F894DEBF0FBECDBFDF91CF911F91A1
:102870000F91FF90EF90DF90CF90BF900C94171ABC
:10288000002319F08B2D817001C08695882309F4EF
:1028900079C1812F829586958770880F880F912F37
:1028A0009F70C92ED12CE12CF12C082E04C0CC0C29
:1028B000DD1CEE1CFF1C0A94D2F714FF12C04FE07F
:1028C00050E060E070E004C0440F551F661F771FA2
:1028D0008A95D2F7CB01BA01609570958095909555
:1028E00003C060E070E0CB012B2D26952695237068
:1028F000422F50E042305105D9F04330510569F183
:102900006C297D298E299F294130510551F1269648
:102910000FB6F894DEBF0FBECDBFDF91CF911F91F0
:102920000F91FF90EF90DF90CF90BF900C94F81A2A
:102930006C297D298E299F2926960FB6F894DEBF33
:102940000FBECDBFDF91CF911F910F91FF90EF9000
:10295000DF90CF90BF900C940A1B0E94F81AC70119
:10296000B60126960FB6F894DEBF0FBECDBFDF913D
:10297000CF911F910F91FF90EF90DF90CF90BF907C
:102980000C94E61A103FD1F128F480E4810F8032D4
:1029900050F0A0C0123F09F462C008F44BC0133FCE
:1029A00009F472C097C0F12FF071FF2E8B2D8F713B
:1029B000002351F00E947F1A812FFF2019F0829589
:1029C000807F68CE8F7066CE0E94A01A812FFF2074
:1029D00019F08295807F01C08F7026960FB6F8940B
:1029E000DEBF0FBECDBFDF91CF911F910F91FF9042
:1029F000EF90DF90CF90BF900C9495120023B1F030
:102A0000253008F0BFC08B2D8F7126960FB6F89435
:102A1000DEBF0FBECDBFDF91CF911F910F91FF9011
:102A2000EF90DF90CF90BF900C94C51A263008F03D
:102A3000A9C0E9CF0023A9F08B2D8F7126960FB680
:102A4000F894DEBF0FBECDBFDF91CF911F910F91E4
:102A5000FF90EF90DF90CF90BF900C947F1A0023EF
:102A600059F38B2D8F7126960FB6F894DEBF0FBEEB
:102A7000CDBFDF91CF911F910F91FF90EF90DF902D
:102A8000CF90BF900C94A01A002399F08B2D8F71DA
:102A900026960FB6F894DEBF0FBECDBFDF91CF9163
:102AA0001F910F91FF90EF90DF90CF90BF900C940B
:102AB0006A1A26960FB6F894DEBF0FBECDBFDF911F
:102AC000CF911F910F91FF90EF90DF90CF90BF902B
:102AD0000C94651A0023A9F0222309F4ADCF812FAD
:102AE00026960FB6F894DEBF0FBECDBFDF91CF9113
:102AF0001F910F91FF90EF90DF90CF90BF900C94BB
:102B0000F711222309F4ADCF812F26960FB6F89442
:102B1000DEBF0FBECDBFDF91CF911F910F91FF9010
:102B2000EF90DF90CF90BF900C9462124B2D4F70BE
:102B3000612FC6010E94071E26960FB6F894DEBFCD
:102B40000FBECDBFDF91CF911F910F91FF90EF90FE
:102B5000DF90CF90BF900C9465194B2D4F70612F73
:102B6000C60126960FB6F894DEBF0FBECDBFDF912B
:102B7000CF911F910F91FF90EF90DF90CF90BF907A
:102B80000C940A1E26960FB6F894DEBF0FBECDBF7A
:102B9000DF91CF911F910F91FF90EF90DF90CF9039
:102BA000BF9008950E94641C0E94331C0E947E1CEA
:102BB0000E94AC200E947A1F80E090E00E945E108C
:102BC00080E090E00C948C100E94541C0C94D21560
:102BD000CF93DF9300D000D01F92CDB7DEB7942FF4
:102BE0004983252F5A836B837C838D834C815D8140
:102BF000452B39F12F3F11F49F3F19F149815A813B
:102C00006B817C818D810E941D1B292F22952F7045
:102C100030E02C30310504F52A3031055CF42250C7
:102C200031092230310568F4853A80F4843090F41B
:102C3000823080F0883E38F4803E60F48450813ADF
:102C400048F080E014C0803FE1F704C090E2980FA4
:102C5000983080F781E00BC02C30310521F493FBD4
:102C6000882780F904C02F303105C9F3EACF0F90CF
:102C70000F900F900F900F90DF91CF910895CF9309
:102C8000DF9300D000D01F92CDB7DEB70F900F902A
:102C90000F900F900F90DF91CF910895CF93DF9316
:102CA00000D000D000D0CDB7DEB726960FB6F8948E
:102CB000DEBF0FBECDBFDF91CF9108951F93CF939D
:102CC000DF93C091CE0116E08091CF01C81799F033
:102CD000D0E01C9FF0011D9FF00D1124E053FE4F2A
:102CE0004081518162817381848195810E944E1659
:102CF0002196C770E9CFDF91CF911F910895409140
:102D000000025091010260910202709103028091D1
:102D10000402909105020C944E1680910502829552
:102D20008F7009F054C080910202882309F44FC0CB
:102D30008091CE01A091CF016091000270910102BB
:102D40004091030250910402B6E08A1709F43FC093
:102D500090E041155105C1F17F3F11F46F3FA1F1A2
:102D6000B89FF001B99FF00D1124E053FE4F21816F
:102D700072132AC02081621327C02281211124C02E
:102D8000238134812417350710F421503109241B85
:102D9000350B283C3105C0F4209105022F702061CD
:102DA0002093050226E0289FF001299FF00D1124B1
:102DB000EB52FE4F80818F708061808380E092E0D3
:102DC0000E949C120C945E1601968770BECF0895E7
:102DD000BF92CF92DF92EF92FF920F931F93CF9308
:102DE000DF93CDB7DEB761970FB6F894DEBF0FBEA5
:102DF000CDBF7C0185E0F701DE011D9601900D92AB
:102E00008A95E1F7D7014C9111965C911197129632
:102E1000DC90129713960D911C911497309100023B
:102E2000609101028091030290910402009709F4DD
:102E300077C16F3F19F43F3F09F472C1B0900202AD
:102E4000BB2009F4C5C0209105020817190728F016
:102E5000F801E81BF90BCF0104C080959095800F15
:102E6000911FCC24C394883C910580F0C12C207F15
:102E700009F0CCC0702F198B088B6D2D89890E94A9
:102E80003F1680E092E00E949C12B6C0822F807FA5
:102E900009F047C0651314C0341312C0D11010C01C
:102EA0002F702061209305020E947F1680E092E03F
:102EB0000E949C1280910502D70115968C932FC019
:102EC0000115110519F15F3F11F44F3FF9F0CD2CB9
:102ED000D1101CC08091CE012091CF0136E0821725
:102EE00009F45CC090E0389FF001399FF00D112487
:102EF000E053FE4F6181561306C06081461303C044
:102F00006281611103C001968770E9CFCD2CDD206D
:102F100009F426C180910502816080930502C12CCD
:102F20001FC1651308C0341306C0D11004C08091BE
:102F30000502D701C9C04D875E87DF86702F198BC8
:102F4000088B6D2D89890E94E8158823E9F1DD2021
:102F5000D9F120910502822F82958F7090E002971F
:102F600074F0809100029091010298878F831986F6
:102F70001B870A872C87CE0107960E949C1286E049
:102F8000F701A0E0B2E001900D928A95E1F70E946E
:102F90008D160E947F16CC24C394E2C0702F198B2B
:102FA000088B60E089890E941D1B292F22952F70B4
:102FB00030E0223031050CF0C7C09F7009F0C1C06D
:102FC000805E883008F4CCC0C7010E949C12E3CF19
:102FD0000817190708F456C0F801E81BF90BCF01D0
:102FE000883C910508F453C0C12C702F198B088BB5
:102FF0006D2D89890E943F16E0E0F2E086E0DF0156
:103000001D928A95E9F70E947F16AAC0651314C025
:10301000341312C0D11010C080910502F7018583CE
:10302000C7010E949C1286E0E0E0F2E0DF011D9201
:103030008A95E9F7CB2C94C04D875E87DF86702F89
:10304000198B088B6D2D89890E94E815882309F456
:10305000BBCFDD2009F4B8CF20910502822F8295E5
:103060008F7090E002970CF48ACF809100029091CB
:1030700001029A8389831B821D830C832E83CE01D8
:1030800001967BCF80959095800F911FA9CFCD2C75
:10309000DD2009F499CF65132EC034132CC0209184
:1030A000050220FD1FC0822F82958F70D9F0D701B5
:1030B00015962C9315978F3049F08F5F982F929526
:1030C000907F822F8F70892B15968C93C7010E9459
:1030D0009C1286E0F701A0E0B2E001900D928A9583
:1030E000E1F791CF86E0F701A0E0B2E001900D9208
:1030F0008A95E1F735C04D875E87DF86702F198B83
:10310000088B6D2D89890E94E815811138CF809137
:103110000502816080930502C7010E949C1220C0B5
:10312000DD2009F451CF4D875E87DF86702F198B24
:10313000088B6D2D89890E94E815882309F444CFF6
:103140001ECF81113DCF0CC0243031050CF03CCF97
:103150009F7009F435CFF7019581907F09F030CF4A
:103160008C2D61960FB6F894DEBF0FBECDBFDF91F8
:10317000CF911F910F91FF90EF90DF90CF90BF9074
:1031800008951F93CF93DF93CDB7DEB72C970FB67B
:10319000F894DEBF0FBECDBF4F83588769877A870B
:1031A0008B879C87CE0107960E94E816882369F0DA
:1031B0008F8198852A853B85232BF1F19F3F09F06C
:1031C00063C08F3F09F060C037C086E0FE013796CC
:1031D000DE01119601900D928A95E1F76F81788555
:1031E000EA85FB85309741F17F3F11F46F3F21F174
:1031F0002091CF0130E0C901019687709927409155
:10320000CE0150E08417950709F447C069837A839B
:10321000FD83EC8396E0929FD001939FB00D112423
:10322000A053BE4FFE01319601900D929A95E1F7A1
:103230008093CF010E945E1616E08091CE0190919E
:10324000CF018917C1F1189FC001112480539E4FEF
:103250000E94E816882379F1E091CE011E9FF001CB
:103260001124E053FE4F408151816281738184813A
:1032700095810E944E168091CE0190E00196877054
:1032800099278093CE01D9CF4F81588569857A855A
:103290008B859C850E944E16CFCF0E94E41510921C
:1032A000CF011092CE01E0E0F2E086E0DF011D9256
:1032B0008A95E9F7C1CF2C960FB6F894DEBF0FBE02
:1032C000CDBFDF91CF911F910895DF92EF92FF92D2
:1032D0000F931F93CF93DF93FC01892B09F48AC0CE
:1032E000E12CF12CDD24D394EF01219684918537D4
:1032F00009F461C058F4843708F04EC0843008F0F7
:103300006AC08130D1F0823071F174C0883709F41D
:103310005DC050F4863709F455C0873709F06AC09C
:103320008E2D0E94511C54C09CE7980F903708F0D6
:1033300061C08F770E94621250C08F010E5F1F4FD5
:10334000FE01849190E2980F983050F48770FD2D23
:1033500001C0FF0F8A95EAF78F2F0E94571C14C0F7
:103360000E94F71113C08F010E5F1F4FFE01C49121
:1033700080E28C0F883060F4C7708D2D01C0880FFB
:10338000CA95EAF70E945D1C0E947E1CE80125C0D8
:103390008C2F0E946212FACF9F012E5F3F4FFE01D9
:1033A000C491CC2369F08FE99FE00197F1F700C049
:1033B0000000C150F6CF9F012E5F3F4FFE01F490F9
:1033C000E9010BC00E94411CE82E07C00E94541C5A
:1033D0000E947E1C02C00E94F7118F2D882341F0AD
:1033E000EFE9FFE03197F1F700C000008150F6CF20
:1033F000FE017ACFDF91CF911F910F91FF90EF9057
:10340000DF9008956093860270938702809388020C
:10341000909389020C94D01C089560938A02709353
:103420008B0280938C0290938D020C94CF1C0F938F
:103430001F9300918A0210918B0220918C0230918F
:103440008D02602B712B822B932B60938A027093D9
:103450008B0280938C0290938D021F910F910C949C
:10346000CF1C0F931F9300918A0210918B02209121
:103470008C0230918D026023712382239323609309
:103480008A0270938B0280938C0290938D021F911D
:103490000F910C94CF1C0F931F9300918A021091EF
:1034A0008B0220918C0230918D0260277127822738
:1034B000932760938A0270938B0280938C0290937F
:1034C0008D021F910F910C94CF1C60E070E0CB0136
:1034D0000C94021A0F931F9341E050E060E070E0FB
:1034E0008A019B0104C0000F111F221F331F8A9500
:1034F000D2F7C901B8011F910F910C94021A0F93D2
:103500001F9341E050E060E070E004C0440F551F9D
:10351000661F771F8A95D2F7809186029091870265
:10352000A0918802B09189028A019B01082B192B76
:103530002A2B3B2BC901B8011F910F910C94021A41
:103540000F931F9341E050E060E070E004C0440F2F
:10355000551F661F771F8A95D2F740955095609545
:1035600070958091860290918702A0918802B09117
:1035700089028A019B01082319232A233B23C901BD
:10358000B8011F910F910C94021A0F931F9341E001
:1035900050E060E070E004C0440F551F661F771FC5
:1035A0008A95D2F78091860290918702A091880235
:1035B000B09189028A019B01082719272A273B27F6
:1035C000C901B8011F910F910C94021A0F931F9318
:1035D0000091860210918702209188023091890221
:1035E000602B712B822B932B1F910F910C94021A3D
:1035F0000F931F93009186021091870220918802F9
:103600003091890260237123822393231F910F91AC
:103610000C94021A0F931F93009186021091870257
:103620002091880230918902602771278227932791
:103630001F910F910C94021A08958F929F92AF924E
:10364000BF92DF92EF92FF920F931F93CF93DF937E
:1036500000D000D01F92CDB7DEB76B837C838D8303
:103660008A018C819D81892B21F01F3F29F44F3FD6
:1036700019F480E090E04CC08B818823C9F18090E0
:103680008A0290908B02A0908C02B0908D02809163
:10369000860290918702A0918802B0918902882ABF
:1036A000992AAA2ABB2A8FE1E82EF12CD501C40160
:1036B0000E2C04C0B695A795979587950A94D2F7D6
:1036C00080FF07C0DE2CB8018E2D0E94DD1D019702
:1036D00029F481E0E81AF10848F7D12C88E0189F16
:1036E000F0011124E00FF11DEA5FFD4FD08209C007
:1036F00088E0189FF0011124E00FF11DEA5FFD4FF3
:10370000D08009831A8369817A818D2D0E94DD1D05
:103710000F900F900F900F900F90DF91CF911F910E
:103720000F91FF90EF90DF90BF90AF909F908F90A0
:10373000089590910A01992321F090910B01911124
:1037400009C020910C0130910D01F90132969FEFD3
:1037500040E030C0982F9695969596959F31A0F4AD
:10376000E0910C01F0910D01E90FF11D877021E04E
:1037700030E0A90102C0440F551F8A95E2F7CA0143
:103780009181892B818308959091B10290FF23C08C
:103790001F928F9389E194E09F938F930E942C0650
:1037A0000F900F900F900F9008959F3F39F04F5F4B
:1037B0004E3141F051915813F8CF0DC05111F7CF50
:1037C000942FF5CF9F3F39F0F901E90FF11D97FDD7
:1037D000FA9582830895089590910A01992321F022
:1037E00090910B01911109C020910C0130910D01B4
:1037F000F9013296205E3F4F30C0982F96959695EE
:1038000096959F31A8F4E0910C01F0910D01E90F1C
:10381000F11D877021E030E0A90102C0440F551F5F
:103820008A95E2F7CA018095918189238183089561
:103830009091B10290FF16C01F928F938BEF93E08F
:103840009F938F930E942C060F900F900F900F90D4
:1038500008953196E217F30729F090819813F9CF74
:103860001082F7CF089581E090E0E0910C01F09193
:103870000D01E80FF91F1082019680329105A9F71A
:1038800008958091B00208959091B002892B8093A1
:10389000B002089580959091B00289238093B00280
:1038A00008958093B00208951092B0020895909107
:1038B000AF02892B8093AF02089580959091AF025B
:1038C00089238093AF0208951092AF0208958093E8
:1038D0008E02089510928E02089580910C019091AD
:1038E0000D01FC0131969C01205E3F4F80E09191DB
:1038F00091118F5FE217F307D1F70895E0910C0162
:10390000F0910D018091B0028083E0910C01F09163
:103910000D0190818091AF02892B808380918E026E
:10392000882361F0E0910C01F0910D019081892BC9
:1039300080830E946D1C811110928E0280910C0177
:1039400090910D010C940A109093390180933801E5
:1039500008958295982F9C7C392F36953695282F7F
:10396000237344E0249FC0011124932F982B292F07
:103970002A7A2695892F8575880F822B08950895B8
:10398000CF93DF9300D000D01F92CDB7DEB70F905A
:103990000F900F900F900F90DF91CF9108950895A1
:1039A00008950C9463118091C602843021F1109225
:1039B000B20220E488E190E00FB6F894A8958093D5
:1039C00060000FBE2093600083B7817F846083BF57
:1039D00083B7816083BF7894889583B78E7F83BFD8
:1039E0000FB6F894A895809160008861809360007C
:1039F000109260000FBE0895CF930E94B5110E94EF
:103A0000AE070E94B611C0E08C2F0E9419088111E8
:103A100004C0CF5FC031C1F701C081E0CF910895EC
:103A20000E941F080C94E4151F920F920FB60F927C
:103A300011248F939F93AF93BF938091B202811112
:103A400013C08091B3029091B402A091B502B091DD
:103A5000B6024196A11DB11D8093B3029093B402AA
:103A6000A093B502B093B602BF91AF919F918F9191
:103A70000F900FBE0F901F90189582E084BD93E0C9
:103A800095BD9AEF97BD80936E0008952FB7F89477
:103A90008091B3029091B402A091B502B091B602A8
:103AA0002FBF08952FB7F8946091B3027091B402BC
:103AB0008091B5029091B6022FBF0895CF92DF9208
:103AC000EF92FF920F931F932FB7F8944091B30298
:103AD0005091B4026091B5027091B6022FBF6A0195
:103AE0007B01EE24FF248C0120E030E0C016D106DB
:103AF000E206F30610F4415051099A01281B390BD4
:103B0000C9011F910F91FF90EF90DF90CF90089522
:103B10001F920F920FB60F9211248F939F93AF9322
:103B2000BF938091B3029091B402A091B502B0917D
:103B3000B6020196A11DB11D8093B3029093B40209
:103B4000A093B502B093B602BF91AF919F918F91B0
:103B50000F900FBE0F901F9018950E940C0DF894B7
:103B60002FEF87EA91E6215080409040E1F700C0B6
:103B7000000087E090EBDC018093CF029093D002AD
:103B8000A093D102B093D2029CE088E10FB6F894E2
:103B9000A895809360000FBE90936000FFCF28E04F
:103BA000929FF0011124E80FF11DE052FF4F949114
:103BB000892F8F7092959F700895CF93C82FCB0156
:103BC0000E94CF1D282F30E080E1989FA001112492
:103BD000422B532B4038510519F480E090E015C07A
:103BE0009770E92FF0E088E0C89FE00DF11D1124E7
:103BF00084E0EE0FFF1F8A95E1F7E20FF31FEE0F4F
:103C0000FF1FE050F84985919491CF91089580E08D
:103C100090E0089508958091B90280FF0BC06091F3
:103C2000110185E0689FB001112475956795759520
:103C300067952BC081FF09C06091110185E0689FE5
:103C4000B00111247595679520C082FF07C060916F
:103C5000110185E0689FB001112417C09091BA024C
:103C60009923D1F060911001961788F720911101E6
:103C700085E0289F90011124929FA001939F500DF1
:103C8000112470E0CA010E94E5256038710540F4F6
:103C90006115710539F002C065E070E0862F089566
:103CA0008FE7089581E008958091B90280FF08C0F0
:103CB00060910F0170E0759567957595679521C0C6
:103CC00081FF06C060910F0170E07595679519C07E
:103CD00082FF04C060910F0170E010C09091BA02A1
:103CE0009923C1F060910E019617A0F780910F0102
:103CF000899FC001112470E00E94E525603871059C
:103D000028F46115710521F0862F08958FE7089535
:103D100081E0089561E070E0F4CF803F21F40E94DB
:103D20000B1E819504C0813F29F40E940B1E8093D5
:103D3000BD020895823F21F40E940B1E819504C0AC
:103D4000833F29F40E940B1E8093BC020895893F93
:103D500019F40E94541E05C08A3F31F40E94541E7B
:103D600081958093BE0208958B3F21F40E94541EDA
:103D7000819504C08C3F29F40E94541E8093BF0299
:103D80000895843F21F48091BB02816017C0853F74
:103D900021F48091BB02826011C0863F21F48091A2
:103DA000BB0284600BC0873F21F48091BB02886016
:103DB00005C0883F31F48091BB0280618093BB02D3
:103DC00008958D3F21F48091B90281600BC08E3F30
:103DD00021F48091B902826005C08F3F29F480915F
:103DE000B90284608093B9020895803F39F48091CC
:103DF000BD0287FF6CC01092BD0269C0813F29F4EB
:103E00008091BD021816BCF362C09091BC02823F43
:103E100029F497FF5CC01092BC0259C0833F19F48B
:103E20001916CCF354C0893F41F48091BE02181694
:103E30000CF04DC01092BE024AC08A3F29F4809116
:103E4000BE0287FF44C0F6CF8B3F39F48091BF029A
:103E500087FF3DC01092BF023AC08C3F29F4809189
:103E6000BF021816BCF333C0843F21F48091BB021B
:103E70008E7F17C0853F21F48091BB028D7F11C0DA
:103E8000863F21F48091BB028B7F0BC0873F21F4DA
:103E90008091BB02877F05C0883F31F48091BB02CF
:103EA0008F7E8093BB0213C08D3F21F48091B902B5
:103EB0008E7F0BC08E3F21F48091B9028D7F05C0AB
:103EC0008F3F29F48091B9028B7F8093B902809152
:103ED000BC0281110EC08091BD0281110AC0809187
:103EE000BE02811106C08091BF02811102C01092F2
:103EF000BA0208958091B10283FF7EC08EE594E0FE
:103F00000E9493058091BB021F928F9389E594E0F4
:103F10009F938F930E942C0687E594E00E9493055F
:103F20008091BC02282F082E000C330B3F938F93F7
:103F300084E594E09F938F930E942C0682E594E0A1
:103F40000E9493058091BD02282F082E000C330B90
:103F50003F938F938FE494E09F938F930E942C065E
:103F60008DE494E00E9493058091BE02282F082ED4
:103F7000000C330B3F938F938AE494E09F938F93CD
:103F80000E942C0688E494E00E9493058091BF0271
:103F9000282F082E000C330B3F938F9385E494E079
:103FA0009F938F930E942C0682E494E00E949305D5
:103FB0008091BA021F928F938FE394E09F938F9327
:103FC0000E942C068DE394E00E9493058091B90233
:103FD0001F928F938AE394E09F938F930E942C0605
:103FE00087E394E00E9493058DB79EB74C960FB679
:103FF000F8949EBF0FBE8DBF8BEB92E00E945310D2
:104000000E94461D9093B8028093B70208951F93B3
:10401000CF93DF938091B7029091B8020E945E1D0A
:10402000AC019091BA02992321F02091120130E065
:1040300006C0209113018AE0289F900111244217A5
:10404000530708F485C08091BC02C091BD02D09195
:10405000BE021091BF02811107C0C11175C0D111FC
:1040600073C0111171C074C09F3F19F09F5F90938E
:10407000BA02181624F40E940B1E8093BC02809191
:10408000BC0287FF05C00E940B1E81958093BC0275
:104090001C1624F40E940B1E8093BD028091BD0269
:1040A00087FF05C00E940B1E81958093BD02609121
:1040B000BC02662331F1C091BD02CC2311F1062E62
:1040C000000C770B880B990B0E94E02423E333E369
:1040D00043E35FE30E9444250E94A8246093BC024E
:1040E0006C2FCC0F770B880B990B0E94E02423E3F5
:1040F00033E343E35FE30E9444250E94A8246093D6
:10410000BD021D1624F40E94541E8093BE028091AD
:10411000BE0287FF05C00E94541E81958093BE0297
:10412000111624F40E94541E8093BF028091BF0296
:1041300087FF05C00E94541E81958093BF02DF91C6
:10414000CF911F910C947A1F9F3F09F08FCF97CF8B
:10415000DF91CF911F910895EBEBF2E085E0DF0155
:104160001D928A95E9F71092BA021092B902089549
:1041700081E896E00E9493051F9281E08F931F9241
:1041800085E08F9383E396E09F938F930E942C06A4
:104190000F900F900F900F900F900F900895833015
:1041A000E9F128F4813061F0823009F10895853019
:1041B00009F462C008F449C0863009F474C0089557
:1041C00080911301262F30E0280F311D2F3F31053C
:1041D00024F4680F6093130103C08FEF80931301E1
:1041E000809113011F928F938CE695E072C08091AD
:1041F0001201262F30E0280F311D2F3F310524F406
:10420000680F6093120103C08FEF809312018091B9
:1042100012011F928F938AE595E05BC08091110196
:10422000262F30E0280F311D2F3F310524F4680F71
:104230006093110103C08FEF8093110180911101F0
:104240001F928F9387E495E044C080911001262F40
:1042500030E0280F311D2F3F310524F4680F6093A3
:10426000100103C08FEF80931001809110011F9205
:104270008F9382E395E02DC080910F01262F30E0CF
:10428000280F311D2F3F310524F4680F60930F0173
:1042900003C08FEF80930F0180910F011F928F93C6
:1042A00089E195E016C080910E01262F30E0280F9D
:1042B000311D2F3F310524F4680F60930E0103C0B8
:1042C0008FEF80930E0180910E011F928F938EEFDE
:1042D00094E09F938F930E942C060F900F900F9065
:1042E0000F900895833081F128F4813059F08230A5
:1042F000D1F00895853009F449C0B8F1863009F449
:1043000056C0089580911301681720F4861B80938E
:10431000130102C010921301809113011F928F9319
:104320008FEE94E054C080911201681720F4861B30
:104330008093120102C010921201809112011F920B
:104340008F938DED94E043C080911101681720F4A4
:10435000861B8093110102C01092110180911101FE
:104360001F928F938AEC94E032C0809110016817FD
:1043700020F4861B8093100102C0109210018091DE
:1043800010011F928F9385EB94E021C080910F0163
:10439000681720F4861B80930F0102C010920F0152
:1043A00080910F011F928F938CE994E010C080914F
:1043B0000E01681720F4861B80930E0102C0109234
:1043C0000E0180910E011F928F9381E894E09F93DC
:1043D0008F930E942C060F900F900F900F900895CE
:1043E000CF93C82F1F928F9386E897E09F938F9368
:1043F0000E942C0681E090E0A0E0B0E0BC01CD017D
:1044000004C0660F771F881F991FCA95D2F70E94B4
:104410000D1A0F900F900F900F90CF910C94E41500
:10442000CF938732A8F58E3108F02BC1803109F483
:104430009FC0F8F4873009F464C0A8F4863009F00E
:1044400024C18091B102817F8E7F8093B1028BE87D
:1044500097E00E94930588E79AE00E94930581E027
:104460008093C1024CC08B30F1F18E3009F46CC0E6
:104470000CC1863109F4B0C020F4813109F4EDC0DB
:1044800004C1893109F491C08B3109F449C0FDC0E0
:10449000883349F150F4893209F4F1C0853309F4C5
:1044A000EEC0873209F0F1C0EAC0833409F4E7C0F6
:1044B00028F48A3308F4E9C08953E4C0883409F049
:1044C000E4C00E94E41587E69AE00E9493052FEF6E
:1044D00083ED90E3215080409040E1F700C0000060
:1044E0000E94AD1D0CC082EB97E05CC08EE49AE0A8
:1044F0000E9493058091B10281608093B102C1E076
:10450000C9C08091B102C82FC17080FFEFCF8AE58A
:104510009AE00E9493058091B102817F8E7F3DC019
:104520009091B10291FBCC27C0F981E0C827892F77
:10453000C0FB81F98093B102CC2319F081E49AE0A9
:1045400027C083E39AE02EC09091B10292FBCC2762
:10455000C0F981E0C827892FC0FB82F98093B1029E
:10456000CC2319F084E29AE013C084E19AE01AC0E7
:104570009091B10293FBCC27C0F981E0C827892F25
:10458000C0FB83F98093B102CC2351F088E09AE01C
:104590000E9493058091B10281608093B1027AC03C
:1045A0008BEF99E00E949305AACF8CEE99E00E94D0
:1045B00093058AEC99E00E94930586E899E00E94B1
:1045C000930589E599E00E9493058FE099E00E94A8
:1045D000930580EE98E0E6CF82ED98E00E94930587
:1045E0000E94FE0F1F928F9388EB98E09F938F930A
:1045F0000E942C0680910A011F928F9381EA98E015
:104600009F938F930E942C068091B6011F928F93E7
:104610008EE898E09F938F930E942C0680910B0167
:104620001F928F938BE798E09F938F930E942C06A5
:104630000E94521D9F938F937F936F9384E698E01F
:104640009F938F930E942C068DB79EB746960FB608
:10465000F8949EBF0FBE8DBF52CF0E94E415C0914B
:104660000B0181E0C827C0930B01CC2329F08AE518
:1046700098E00E9493050EC08FE498E093CF80E00D
:1046800001C08D510E94F0213ACF8DE498E00E9444
:104690009305C0E08C2FCF91089580E0089580E0CD
:1046A0000895CF93C82F8091C102813079F020F016
:1046B000823009F44DC044C1E0910C01F0910D012C
:1046C00080818152823008F03DC108C0E0910C0128
:1046D000F0910D0180818152823060F48C2F0E9414
:1046E0004D23811104C08C2F0E9410222FC081E025
:1046F00090E02CC08C2F0E944F23811126C0C43122
:10470000E1F070F4CB3081F0C031D1F40E94B820D8
:104710008EE797E00E94930582E08093C10215C066
:10472000C93259F0C83361F48BE897E00E949305D1
:1047300082E897E00E94930508C01092C10204C16C
:104740008CE797E00E949305FFC081E08170FEC076
:10475000C43228F5CE3108F0C1C0CB30A1F1D0F47D
:10476000C73009F0D3C08EE18093130182E38093B8
:1047700012018AE08093110184E18093100188E0A6
:1047800080930F0188E280930E0182E296E00E94FE
:104790009305BFC0C33149F1C431C1F0B7C0CB34B8
:1047A00009F4A9C028F4C93289F0C83361F0AEC059
:1047B000C13509F49EC0C23509F499C0CE3409F060
:1047C000A5C06AE09EC00E94B820A3C08091C0022C
:1047D000882319F01092C0029CC08FE296E00E94DC
:1047E000930581E08093C102B1C089E096E00E9408
:1047F000930587EF95E00E949305809113011F9226
:104800008F9384EF95E09F938F930E942C0682EF05
:1048100095E00E94930580EE95E00E9493058091BB
:1048200012011F928F938DED95E09F938F930E94BD
:104830002C068BED95E00E9493058CEC95E00E9490
:104840009305809111011F928F9389EC95E09F93BE
:104850008F930E942C0687EC95E00E94930586EBCF
:1048600095E00E949305809110011F928F9383EB36
:1048700095E09F938F930E942C0681EB95E00E9418
:1048800093058CE995E00E94930580910F011F929A
:104890008F9389E995E09F938F930E942C0687E977
:1048A00095E00E94930580E895E00E949305809131
:1048B0000E011F928F938DE795E09F938F930E9437
:1048C0002C068BE795E00E9493058DB79EB748961E
:1048D0000FB6F8949EBF0FBE8DBF1BC0CE51EC2FFC
:1048E000F0E0E25DFE4F80818093C00212C061E083
:1048F00003C061E006C06AE08091C0020E94CF2040
:1049000008C08091C0020E94722103C080E296E03C
:1049100013C08091C002882369F01F928F938AE1AF
:1049200096E09F938F930E942C060F900F900F900C
:104930000F9004C087E196E00E94930581E006C0D5
:104940001092C10280E002C080E000CFCF910895B4
:104950000E94AF246894B1110C943E2508950E94E2
:10496000232588F09F5798F0B92F9927B751B0F0B9
:10497000E1F0660F771F881F991F1AF0BA95C9F7E3
:1049800014C0B13091F00E943D25B1E008950C941F
:104990003D25672F782F8827B85F39F0B93FCCF3D2
:1049A000869577956795B395D9F73EF49095809560
:1049B000709561957F4F8F4F9F4F0895E89409C080
:1049C00097FB3EF490958095709561957F4F8F4F42
:1049D0009F4F9923A9F0F92F96E9BB279395F69558
:1049E000879577956795B795F111F8CFFAF4BB0FD6
:1049F00011F460FF1BC06F5F7F4F8F4F9F4F16C03A
:104A0000882311F096E911C0772321F09EE8872FC3
:104A1000762F05C0662371F096E8862F70E060E07F
:104A20002AF09A95660F771F881FDAF7880F9695F8
:104A3000879597F9089557FD9058440F551F59F0E1
:104A40005F3F71F04795880F97FB991F61F09F3F7B
:104A500079F087950895121613061406551FF2CFA4
:104A60004695F1DF08C0161617061806991FF1CFF4
:104A700086957105610508940895E894BB2766271B
:104A80007727CB0197F908950E9457250C94C825E4
:104A90000E94BA2538F00E94C12520F0952311F01C
:104AA0000C94B1250C94B72511240C943E250E943A
:104AB0001B2570F3959FC1F3950F50E0551F629F22
:104AC000F001729FBB27F00DB11D639FAA27F00D67
:104AD000B11DAA1F649F6627B00DA11D661F829F8E
:104AE0002227B00DA11D621F739FB00DA11D621F73
:104AF000839FA00D611D221F749F3327A00D611D90
:104B0000231F849F600D211D822F762F6A2F112471
:104B10009F5750409AF0F1F088234AF0EE0FFF1FA4
:104B2000BB1F661F771F881F91505040A9F79E3FFB
:104B3000510580F00C94B1250C943E255F3FE4F3C1
:104B4000983ED4F3869577956795B795F795E79551
:104B50009F5FC1F7FE2B880F911D9695879597F95A
:104B6000089597F99F6780E870E060E008959FEFEF
:104B700080EC089500240A941616170618060906F4
:104B8000089500240A9412161306140605060895C3
:104B9000092E0394000C11F4882352F0BB0F40F44B
:104BA000BF2B11F460FF04C06F5F7F4F8F4F9F4F8B
:104BB0000895991B79E004C0991F961708F0961B79
:104BC000881F7A95C9F78095089597FB072E16F4EC
:104BD000009407D077FD09D00E94FF2507FC05D07F
:104BE0003EF4909581959F4F0895709561957F4F04
:104BF0000895EE0FFF1F0590F491E02D0994AA1B74
:104C0000BB1B51E107C0AA1FBB1FA617B70710F0B7
:104C1000A61BB70B881F991F5A95A9F780959095E9
:0A4C2000BC01CD010895F894FFCF08
:104C2A0028081909F608C2088E0801018F02280807
:104C3A00140A321E404D36223963031603E002BEBF
:104C4A00028502F80111022A0243026302000102EC
:084C5A00030405060708090028
:106800008800EA44E944E244040005000600070069
:10681000080009000A000B000C000D000E000F001C
:1068200010001100120013001400150016001700CC
:10683000180019001A001B001C001D001E001F007C
:10684000200021002200230024002500260027002C
:10685000280029002A002B002C002D002E002F00DC
:10686000300031003200330034003500360037008C
:10687000380039003A003B003C003D003E003F003C
:1068800040004100420043004400450046004700EC
:10689000480049004A004B004C004D004E004F009C
:1068A000500051005200530054005500560057004C
:1068B000580059005A005B005C005D005E005F00FC
:1068C000600061006200630064006500850067008D
:1068D000680069006A006B006C006D006E006F005C
:1068E0007000710072007300890087008A008B00BD
:1068F000E000E100E200E300E400E500E600E7007C
:00000001FF
